:0200000088294D
:08000800DF00030E8312B400B7
:0E0010000A0EB500040EB6008A110A12B929B4
:100020000330D107D10CD10C7F30D1050000D10BAA
:1000300016280800D008031D1E280800F930FF3ECE
:10004000031D1F280000D00B1E280800D201D30179
:10005000D601D701D40110305405D500D508031DB1
:1000600008000310D60DD70DCE0DCF0DD20DD30D38
:1000700051085302031D3E2850085202031C472812
:100080005008D2025108031CD303D3025614D40AD9
:100090002B28CF014E084F020318080064000130DE
:1000A000D0001A20CF0A4A285008840052080004C1
:1000B000D400540880004E08840052080005D40083
:1000C0005308D500031908000310D40CD503622887
:1000D0004F08FF3C0318500803197728FF30D10060
:1000E0001020FF30CF02D008031CD00368284F082F
:1000F000003C03185008031908004F08D1001020D5
:100100000800073083129900C030831681008312E3
:10011000C701033047020318BC28C80164304802F5
:100120000318B7280130CE00831605118312CE08BC
:1001300003199E28043005048500A128FB3005051D
:1001400085000130CE004920CE01831605118312AF
:10015000CE080319AF28043005048500B228FB300F
:10016000050585000130CE004920C80A8E28FA30E6
:10017000CE004920C70A8928C901FA30490203186C
:10018000E6280130CE00831605118312CE0803192C
:10019000CD28043005048500D028FB3005058500F6
:1001A0000130CE004920CE01831605118312CE08FE
:1001B0000319DE28043005048500E128FB3005051D
:1001C00085000130CE004920C90ABD28FA30CE0092
:1001D00049200130CE00831685128312CE08031900
:1001E000F528203005048500F828DF300505850056
:1001F0009630D1001020CE01831685128312CE08CE
:10020000031906292030050485000929DF3005057A
:100210008500CA010C304A02031822290030CF00A1
:100220000530CE000030D1008530D0001030D20033
:100230000430D30054205408CC004C084B07CB00AA
:10024000CA0A0A294B08CD00CB014D08003C03180F
:1002500083299030CE000130CF004D08D000D1016D
:1002600026205608B9005708BA009630B907031877
:10027000BA0ABB01BC010130CF00831605118312FD
:10028000CF08031947290430050485004A29FB30AB
:10029000050585003908CF003A08D0006820CF0155
:1002A000831605118312CF0803195A290430050457
:1002B00085005D29FB30050585003908CF003A0827
:1002C000D00068203908BB073A08CF003C08031863
:1002D000CF0ACF073908BB073A08D0004F080318E8
:1002E000D00AD0075008BC00CE0111303C02031DDB
:1002F0007B2930303B02031CCE0ACE08031D3B296C
:10030000BB01BC0186290630CE004920CD01E92879
:10031000D5308312A000C430A100BB30A200DC3075
:10032000A300A401A501A601A701A801A901AA0192
:10033000AB01AC01AD01AE01AF01C001C101B7011C
:10034000B801C201C301C401C501B001B101B201CC
:10035000B301BE01BF01BD01C601E830B9000330E1
:10036000BA00BB01BC01CB01CC01CD018A110A123C
:1003700081288312360E8400350E8A00340E8300E5
:06038000DF0E5F0E090014
:02400E00940F0D
:00000001FF
